:02000000232AB1
:10000800A000030EA100E130831281000B11070844
:10001800B8030319F339B9030319CF39BB0303191B
:10002800FC3983128700BA0303190511BC030319AD
:100038002220210E8300A00E200E09001F30BC00D4
:10004800A2013408B800B81F2B28B809B80A031051
:10005800B80CB80803193528B41F342822153528D8
:10006800A2153508B900B91F3B28B909B90A031008
:10007800B90CB90803194528B51F44282216452884
:10008800A2163708BB00BB1F4B28BB09BB0A0310CD
:10009800BB0CBB0803195528B71F54282214552830
:1000A800A2143608003CBA00B61FBA010310BA0CF5
:1000B800BA080319622883120515642883120511EA
:1000C8002208831287000800A6008A0126088207F2
:1000D800A234A834AE34A634AC34A434A634A6343E
:1000E800A734A6008A0126088207553455345534AA
:1000F80055345534553455348D34BE34A800280849
:10010800A9002608AA002708AB008312851005104D
:100118008512A90803199C288312AB1F0510AB1B75
:1001280005140310AA0DAB0D8514A90385108D289D
:100138008312851605142E19051008000830A4002E
:10014800A501A4080319B228831285140310A50D6C
:10015800251085192514A4038510A528250808004D
:100168001030FF0083128714FF080319C92883126F
:10017800AF1F0710AF1B07140310AF0D2F10B01BD4
:100188002F140310B00DFF03B8288312871007102F
:1001980008002F08FF001030FF0083120515FF0824
:1001A80003191529831287017F08013A0319E928E1
:1001B800043A0319EF28033A0319F528053A0319F5
:1001C800FB28013A0319012907298312AF1F0710D9
:1001D800AF1B07140C298312AF1F8710AF1B87149E
:1001E8000C298312AF1F0711AF1B07150C298312A7
:1001F800AF1F8711AF1B87150C298312AF1F07127A
:10020800AF1B07160C298312AF1F8712AF1B871667
:100218000310AF0D2F10B01B2F140310B00DFF03E8
:10022800D32883120511870108000330B300320870
:1002380031060319302983169B0132089A001C15D0
:1002480055309D00AA309D009C1483128C1F2929CB
:1002580083128C1383161C11E130831281000B1159
:100268008B178B16080024102F08013A0319492907
:10027800043A03195229033A03195629053A03196E
:100288005A29013A03195E296129300B612933087B
:10029800033A031961291921241461292414300807
:1002A800B400612924143008B500612924143008E9
:1002B800B700612924143008B600241C71292410C1
:1002C8003308023A031919213308033A031D712927
:1002D8002B3083128E00CF308F0008008530A600A7
:1002E800CE30A700103082208730A600CE30A7007D
:1002F800103082288312851005108512A220A300D1
:10030800231F8829A301AE14231A2E15A31F9A2987
:10031800A220A300A220A3002E1896292E14230899
:10032800AF009A292308B000AE14372183120510B4
:100338008516AE1CA2292E10AE1072290800A30043
:10034800063023020318AF299B30A6009C30A70073
:1003580010308220B5299B30A6009C30A7001030B1
:10036800822023086820A50023087520A4002408FB
:10037800A6002508A70010308220722907308312B2
:10038800990085018701183083168500870183123B
:100398008516083083168100203084008001840A85
:1003A80060300402031CD22983169B011C141A080E
:1003B800B1003108B200093032020318B20111301D
:1003C800831290008E018F010C1083120C1CE929F6
:1003D8004030A600C030A700103082203208A32188
:1003E8000630A600C230A700103082206C30A6006C
:1003F800C430A700103082205530A600C830A700AE
:10040800103082200730A600C630A70010308220A6
:100418004130A600C030A70010308220831281012D
:100428000B110B1D152A8530A600CE30A700103001
:1004380082208730A600CE30A70010308228FF2304
:1004480083169000C2213130831290002B308E0029
:10045800CF308F000C102030B4000A30B500F030D7
:10046800B600E030B700192183120C1C682A2B3023
:100478008E00CF308F000C10330803194D2A013A33
:100488000319532A033A0319592A013A0319612A0D
:10049800682A0130B300B2013208A321682A320861
:1004A800083A031D592A0230B300B20A0930320251
:1004B8000318B2013208A321682A831205118701A3
:1004C800B401B701B501B6018312051A382A7E2195
:0204D800382AC0
:02400E00C401EB
:00000001FF
